:020000040000FA
:06000000852841302A3082
:08000800A000030EA100831209
:100010000C1C2328DD1B23288E015C1C15285C107A
:100020005A088F005D0985051B285C145B088F004A
:100030005D088504DC170C108B180828210E83003E
:10004000A00E200E090005192B2883160117831214
:10005000B23081005D288316011383120B193728F3
:10006000AE17280A03192E17AE1948285628AE13C2
:10007000AE1945282E1F5628AE1A5628A701A601EC
:10008000A501A801AE01AE165D28F030AE055D28D1
:100090002D152E13AE122708AB002608AA0025083E
:1000A000A9002808AC00F030AE055D282E0DA80D83
:1000B000A50DA60DA70DAE1AAE0A8B100B11210EC1
:0800C0008300A00E200E0900D0
:06010A002030840080019A
:10011000840A60300402031C872863228316FF23AD
:100120009000831283160C308505870183128501A8
:100130008701073099000030831691009F008312D9
:10014000C83083168100831201309000013083167D
:100150008C00831210308B00BD1BB028851DF72248
:100160003D1BBE013D1BBF013D1FEF2281018E01E2
:100170008F010B118B100B108C130C138C110C10A6
:100180000B178B17D4202D19D6203722B30BD0286C
:10019000031085190314BA0DF0303A020319B02187
:1001A000DC1829233723C2286400080029083F3CB3
:1001B0000319E2282B082A0629062C02031D2D11FB
:1001C000031D08002D110130B7008B1320303707B5
:1001D00083169B001C141A088312A40010303707E2
:1001E00083169B001C141A088312A30000303707E3
:1001F00083169B001C141A088312A2008B17240874
:100200002B02031DAA2923082A02031DAA29013053
:1002100003303702031D3A2929083F3C03192429DA
:1002200040302906E039031D1A293F1F1A293F13C0
:10023000AD17282960302906E039031D28293F1B06
:1002400028293F17AD172829AC1F3F13AC1B3F17B8
:1002500080302906F039031D3129BF1F3129BF1312
:10026000AD1790302906F039031D3A29BF1B3A29F2
:10027000BF17AD17A91FAA29291BAA2922082906D9
:10028000F039A91EE039031DAA29220829050F39D2
:100290000319772901303702031D53293E185329CA
:1002A0003E14AD177D2202303702031D5C29BE18B3
:1002B0005C29BE14AD17912203303702031D652956
:1002C0003E1965293E15AD17A52204303702031DDE
:1002D0006E29BE196E29BE15AD17B9220530370239
:1002E000031D77293E1A77293E16AD17CD2229091D
:1002F00022050F390319AA2901303702031D852968
:100300003E1C85293E10AD17D72202303702031D4F
:100310008E29BE1C8E29BE10AD17DA22033037029B
:10032000031D97293E1D97293E11AD17DD2204308C
:100330003702031DA029BE1DA029BE11AD17E12261
:1003400005303702031DA9293E1EA9293E12AD170B
:10035000E522AA29B70A0630370203180800E52863
:100360000B13DD17B601B3019630B4000130B500B0
:100370000130B70085018701AD131C22D420B30BD7
:10038000DB29031085190314BA0DF0303A02031962
:100390000A2AB41F8501B41F8701B40BDB29370873
:1003A000B6080319B6000319D929FF308500870064
:1003B000B6039630B4002D1DBE292D11A91FBE29EC
:1003C000291BBE29A91E29120F3029050319BE2990
:1003D000B9012918B90AA918B90A2919B90AA91914
:1003E000B90AB918BE293919BE298B13203037072D
:1003F000BC002B08BB00452210303707BC002A0880
:10040000BB00452200303707BC002908BB0045224D
:100410008B17162285018701B70AB601063037020D
:10042000031CBE290B17DD13EF220800053037022D
:1004300003190800850187011430B90033308F1F7C
:1004400085008F1B8501D4202D1D1E2A2D11290A00
:1004500003192E2AA91F1E2A291B1E2A0F3029051F
:10046000031D1C2AB90B1E2A850187010800AD1F38
:100470000800AD131030BC003E08BB0045223030F0
:10048000BC003F08BB00452208003C088B138316C4
:100490009B001C141A0883128B173B0203190800D7
:1004A0008B133B0883161C159A003C089B005530A3
:1004B0009D00AA309D009C1464009C185C2A1C11AD
:1004C00083128B1708000A30DE007D30DF008316B0
:1004D00000309B001C141A088312BD0083161030D4
:1004E0009B001C141A088312BE00831630309B0038
:1004F0001C141A088312BF0008000730C100D21074
:100500000E303E05031D08008B13831620309B0020
:100510001C141A088312D6008B178E018F010C1041
:1005200008000630C20052110D303E05031D0800C0
:100530008B13831620309B001C141A088312D600DC
:100540008B178E018F010C1008000730C300D211E9
:100550000B303E05031D08008B13831620309B00D3
:100560001C141A088312D6008B178E018F010C10F1
:1005700008000530C400521207303E05031D080074
:100580008B13831620309B001C141A088312D6008C
:100590008B178E018F010C1008008B1383164030CF
:1005A0009B001C141A088312D1008B1708008512B7
:1005B000DD12080005125D120800DC1C8510DD103C
:1005C0000800DC1C05105D1008008B1383164130F9
:1005D0009B001C141A088312D1008B170800C1015C
:1005E000C201C301C4013E1EE52ACD2A0800B6019E
:1005F000B301B4013D1CFF2A3D10BD140C2BBD1CE2
:10060000042BBD103D150C2B3D1D092B3D11BD15B7
:100610000C2BC030BD053D143D083F39B6006400C9
:10062000112B122B132B142B152B3330B41B8500DD
:10063000B41F8501B30B0F2BB40B0F2B0310B60C9B
:10064000B608031D0F2B0030BC003D08BB0045223F
:100650000800BF1F342B3F1B85103F1B05143F1F95
:1006600085143F1F05100800851005100800DC10D8
:10067000BD18DC14BD19DC145108FF3CDB00F03060
:100680005107DA000F303E0503190800D608031998
:10069000522BDC1F0800DC13DF0B08007D30DF006D
:1006A000D60308003E1CDD123E18DD16BE1C5D128E
:1006B000BE185D163E1DDD10DC18602B3E19DD14E2
:1006C000BE1D5D10DC18662BBE195D14DC185D10B4
:1006D000DC18DD10DE0B08000A30DE00521C85122B
:1006E000D21C0512DC18782B521D8510D21D051066
:1006F0003D187F2BBD187F2B0F30D20008008123BF
:1007000008004D08D500DC23CD004E08D500DC23C1
:10071000CE004F08D5004D1CDC23CF005008D5007B
:10072000CD1CDC23D000C108031952140319A42BDB
:10073000C90BA42BCD1BC1034D08C900CD18521401
:10074000CD1E5210CD1D5210C2080319D214031928
:10075000B52BCA0BB52BCE1BC2034E08CA00CE1A4E
:10076000D2144E1DD2104E1FD210BD18DB2BBD1956
:10077000DB2BC308031952150319CA2BCB0BCA2B49
:10078000CF1BC3034F08CB004F1A52154F1F5211F6
:10079000CF1D5211C4080319D2150319DB2BCC0B42
:1007A000DB2BD01BC4035008CC00501AD215D01F2D
:1007B000D211D01DD2110800C001D5080319D503EC
:1007C00055184014D51A40144008C001551C401457
:0C07D000D51E4014C005C00C550C0800DC
:084000000700000006000200A9
:02400E00CC01E3
:1042000001008100820084008800B100B200B40087
:10421000B800A100A200FF00FF00FF00FF00FF00A8
:104220000000010001000100010001000100010087
:10423000010001000100FF00FF00FF00FF00FF0080
:10424000000000000000000000000000000000006E
:10425000000000000000FF00FF00FF00FF00FF0063
:104260000000FF00FF00FF00FF00FF00FF00FF0055
:10427000FF00FF00FF00FF00FF00FF00FF00FF0046
:1042800002000F00FF00FF00FF00FF00FF00FF0023
:10429000FF00FF00FF00FF00FF00FF00FF00FF0026
:1042A000FF00FF00FF00FF00FF00FF00FF00FF0016
:1042B000FF00FF00FF00FF00FF00FF00FF00FF0006
:1042C000FF00FF00FF00FF00FF00FF00FF00FF00F6
:1042D000FF00FF00FF00FF00FF00FF00FF00FF00E6
:1042E000FF00FF00FF00FF00FF00FF00FF00FF00D6
:1042F000FF00FF00FF00FF00FF00FF00FF00DD00E8
:00000001FF
